:020000040000FA
:100000000528000000000000AA2A192026208020D0
:100010003A2048202F2058205B2078228C22E5208F
:1000200046211D213E22522291202F203321B8202B
:10003000A92285018316FF3085008312860183166D
:100040005F308100FF308600831208005F30A0001F
:10005000213084008001840AA00B2A28080018306F
:10006000A10030308400000807398000840AA10B09
:10007000332808001830A0003030840086193E284C
:10008000861D402806088000840AA00B3E28080030
:100090000830A0000E30A1003230840000192C146A
:1000A000A119AC0D03308407A103A00B4E28080052
:1000B0006008A60008000830A000A101A201A30169
:1000C0003030230784000008A800A30A840A800DAA
:1000D000800D800D0008A807A30A840A800D800DFA
:1000E000800D800D800D800D0008A807603022076C
:1000F000840028088000A30AA20AA00B6028080038
:100100001030A000A10121080A148A148123A8003C
:1001100050302107840028088000A10AA00B832802
:100120000800A0010830A100A20168302007840067
:100130000008A80030302207840028088000A20AA6
:10014000A80CA80CA80C2808303022078400280826
:100150008000A20AA80CA80CA80C2808303022079E
:10016000840028088000A20AA00AA10B9528080094
:10017000A0011830A10086018316F030860083129A
:100180003030200784000008860080150008000039
:100190000000000000000000000000008600A00A2F
:1001A000A10BC028000000000000000000000000BB
:1001B00086010000000000000000000000000000B8
:1001C0008316FF308600831208000830A1000E302D
:1001D000A20060308400AB010930A0000008A80034
:1001E000AA012808AA06A80DA00BF1282118F828B2
:1001F000AA1B2B14FD28AA1F2B14A219AB0D840ACD
:10020000A203A10BEC28080083160F30860083128E
:100210002B08A800A80DA80DA80DA80D2808860079
:1002200083160F30860083122B08A800A80CA80C98
:10023000A80CA80C2808850008000730A100683029
:100240008400AB010930A0000008A800AA0128081A
:10025000AA06A80DA00B27292A182B14AB0D840A77
:10026000A10B222908000830A000473084002B1879
:100270000015AB0C03308402A00B372908002C08B2
:100280002B063F39031D4529080045290730A000EA
:10029000A101A9016008213A031992296008223AB4
:1002A000031992296008233A031992296008413AF8
:1002B000031984290730A1076008423A03198429E9
:1002C0000730A1076008433A031984290730A107C2
:1002D0006008443A031984290730A1076008613A8D
:1002E000031984290730A1076008623A0319842999
:1002F0000730A1076008663A031984290730A1076F
:1003000060086B3A031984290A148A146130840046
:10031000210800230006031D9529840AA10AA003D1
:10032000031D88296008A90095290830A000A101B3
:100330002908213A031DA7295030A5000730A30042
:10034000A0192B220A148A1421083923212A2908EA
:10035000223A031DB6295730A5000730A300A01983
:100360002B220A148A1421084223212A2908233A1D
:10037000031DC5295E30A5000230A300A0192B2261
:100380000A148A1421084B23212A2908413A031D03
:10039000CE290A148A142108BE23212A2908423AA8
:1003A000031DD7290A148A142108CE23212A2908DB
:1003B000433A031DE0290A148A142108D823212A6C
:1003C0002908443A031DE9290A148A142108E8235C
:1003D000212A2908613A031DF2290A148A142108E6
:1003E0005423212A2908623A031DFB290A148A147E
:1003F00021085D23212A2908663A031D042A0A14CC
:100400008A1421086623212A29086B3A031D0D2A24
:100410000A148A1421086F23212A0A148A14210835
:1004200078236008D7006108D5006208D30063080C
:10043000D1006408D6006508D4006608D2006708B9
:10044000D000A80068302107840028088000A10A95
:10045000A00B982908006130A4008400A2000008C5
:10046000A8002508840028088000220884000130A4
:10047000A507040AA40AA30B2D2A08000830A0002F
:100480006830A1005830A200220884000008A800AB
:100490002108840028088006A10AA20AA003031DDF
:1004A000442A08002908663A0319692A0830A0007E
:1004B0006830A1005030A200220884000008A80083
:1004C0002108840028088007A10AA20AA003031DAE
:1004D0005C2A0800220884000008A8002108840083
:1004E00028088002A10AA20AA003031D5C2A0800B2
:1004F0000830A0006030A1005030A2002208840023
:100500000008A8002108840028088002A10AA20A85
:10051000A003031D7E2A08000830A0006030A1005F
:100520005830A200220884000008A8002108840096
:1005300028088006A10AA20AA003031D922A080027
:100540000430B5000430BB000430C1000430C700E3
:10055000080008280900000000000000000000005A
:10056000000000000000000000000000000000008B
:10057000000000000000000000000000000000007B
:10058000000000000000000000000000000000006B
:10059000000000000000000000000000000000005B
:1005A000000000000000000000000000000000004B
:1005B000000000000000000000000000000000003B
:1005C000000000000000000000000000000000002B
:1005D000000000000000000000000000000000001B
:1005E000000000000000000000000000000000000B
:1005F00000000000000000000000000000000000FB
:1006000082074B344534593443344F3444344534F1
:100610006B346534793463346F3464346534313425
:100620007334743472346434663430343134733433
:1006300074347234643466343134743465347334ED
:1006400074347034693463347334653463345F34C0
:100650007634653472344E3461346F346D346934B9
:1006600047344434613469346A3479346F34213422
:100670003F3482073034443449344D344D344934A6
:100680004434303482073134443449344D344D34A9
:1006900049344434313482073234443449344D349B
:1006A0004D34493444343234820737345434453479
:1006B000533454345F344F344B3482073834563417
:1006C00045345234303430343034313482073F349E
:1006D0004834653472346534493461346D3482078A
:1006E0003A3470341F3471341F3400340034013410
:1006F00082075A344534523452344F3452343034F1
:10070000303482074E3441344F344D344934473409
:10071000443452344F344D345334593453345434B4
:1007200045344D34000000000000000000000000CF
:1007300000000000000000000000000000000000B9
:1007400000000000000000000000000000000000A9
:100750000000000000000000000000000000000099
:100760000000000000000000000000000000000089
:100770000000000000000000000000008207333489
:1007800000340034003400340034003400340000FD
:100790000000000000000000000000008207343468
:1007A0000034000000000000000000000000000015
:1007B000820735344134423443342E344234493490
:1007C0004E340000000000000000000000000000A7
:1007D00082073634003400340034003400340034EE
:1007E00000340000000000000000000000000000D5
:1007F00000000000000000000000000000000000F9
:1008000000000000000000000000000000000000E8
:1008100000000000000000000000000000000000D8
:1008200000000000000000000000000000000000C8
:100FF00000000000000000340034FF3FFF3FFF3FCF
:10420000FF00FF00FF00FF00FF00FF00FF00FF00B6
:10421000FF00FF00FF00FF00FF00FF00FF00FF00A6
:10422000FF00FF00FF00FF00FF00FF00FF00FF0096
:10423000FF00FF00FF00FF00FF00FF00FF00FF0086
:10424000FF00FF00FF00FF00FF00FF00FF00FF0076
:10425000FF00FF00FF00FF00FF00FF00FF00FF0066
:10426000FF00FF00FF00FF00FF00FF00FF00FF0056
:10427000FF00FF00FF00FF00FF00FF00FF00FF0046
:10428000FF00FF00FF00FF00FF00FF00FF00FF0036
:10429000FF00FF00FF00FF00FF00FF00FF00FF0026
:1042A000FF00FF00FF00FF00FF00FF00FF00FF0016
:1042B000FF00FF00FF00FF00FF00FF00FF00FF0006
:1042C000FF00FF00FF00FF00FF00FF00FF00FF00F6
:1042D000FF00FF00FF00FF00FF00FF00FF00FF00E6
:1042E000FF00FF00FF00FF00FF00FF00FF00FF00D6
:1042F000FF00FF00FF00FF00FF00FF00FF00FF00C6
:02400E005D1E35
:08400000FF3FFF3FFF3FFF3FC0
:00000001FF
